:030000000219FDE5
:03000B000200AA46
:03002B0002015679
:03005B000202E8B6
:030073000202D5B1
:1000800002030406080C10182030406080040608A3
:100090000C10182030406080A0C00003070F1F0D17
:1000A0000D0403060D0502030202C2AFC0D0C0E07A
:1000B000206214E5256009E473E525F4F58AD2622F
:1000C000D0E0D0D0D2AF3285268AC262E526F46075
:1000D00029D0E0D0D0D290D291D292D2AF32D29069
:1000E000D291D292206F0C206509740AD5E0FDE50B
:1000F0007B4290D0E0D0D0D2AF32758A00C28DD290
:100100006201F301B9306805206502C29001B9307F
:100110006805206502C29101B9306805206502C2F8
:100120009201B9C29330680A2065077428D5E0FDB2
:10013000C29001B9C29430680A2065077428D5E0DE
:10014000FDC29101B9C29530680A2065077428D5AF
:10015000E0FDC29201B9C2AFC2AD53E6EFC0D0C05C
:10016000E0D2D3D2AFC2CEE52A600720744F152A61
:1001700021BD7800790020742EE580307E01F430B6
:10018000E70278FF53DACF207E0343DA20307E0384
:1001900043DA10C2D8C271E580307E01F430E70244
:1001A00079FFC3E89970CB306103752A402074034E
:1001B000752A40885CD270E86003755F0020740D7A
:1001C000E52B6004152B21CD43DA01C2D820700243
:1001D00021E0A85C206102C27020740221DE882226
:1001E0007882B6040385222420CF0AD0E0D0D04301
:1001F000E610D2AD32C2CF053A7802E52A6005306A
:100200007402152AC3E55C94014005755F00412125
:10021000756000756900E55F2401F55F5003755F47
:10022000FF7982B7020D306E1DC3E522943240166D
:10023000854C227982B7030E306E0BC3E5229432CF
:100240004004798E8722C3E5239522600840041577
:100250002341550523D8CA0569E56970021569D59A
:100260006A69756A017808E56B60497805C3E569D4
:10027000956B4057C3E569956C50087801756A0322
:1002800002028FC3E569956D50057801756A01C357
:10029000E5629524401E7982B7040241C0206E14A5
:1002A000852462E569046003856B69756A017523BD
:1002B0003C0202CBE5622850057562FF41C0F56241
:1002C000E5620470067560FF7569FFD0E0D0D04329
:1002D000E610D2AD32C2AF53E67F7592FA7593FF46
:1002E000C260759104D2AF32C2AF53E6EFC2ADC067
:1002F000D0C0E0C0F0D2D3D2AFA8FBA9FCC2D830A6
:100300007102614F53DACF207E0343DA10307E034F
:1003100043DA20D271E580307E01F420E7026126C5
:1003200088278928A13453DACF207E0343DA20308E
:100330007E0343DA10C2D8C271307402A120780063
:10034000E580307E01F430E702A120885CA10853EB
:10035000DACF207E0343DA20307E0343DA10C27105
:10036000206102812853DACF207E0343DA10307EE9
:100370000343DA20C2D8D27188578958C3E895550B
:10038000F8E99556F97B007E087A00C3E8948CE979
:1003900094005005755B00811A882178A2E6A82197
:1003A0006055C3E894C8E994005008E4D2E4FB7AAD
:1003B0000A61F5C3E89468E994015008E4D2E3FBCC
:1003C0007A0F61F5C3E894D0E994025008E4D2E2D0
:1003D000FB7A1E61F5C3E894A0E994055008E4D2C5
:1003E000E1FB7A3C61F5C3E89498E994085008E48D
:1003F000D2E0FB7A787E00C3E89559FCE9955AFD76
:1004000030E70AECF42401FCEDF43400FD755B00E8
:10041000C3EC9AED9E5003755B018859895A855744
:10042000558558567802A108C3E89527F8E995281C
:10043000F9307C0281EC307B0281EC307A0281E57C
:10044000207502814BE9FDE8FC816AE9C313F9E8F4
:1004500013F830790281E5E9C313F9E813F830782D
:100460000281E5E9C313FDE813FC20612CC3EC9481
:0F0470001CED940240028181ED701EC3EC94C814
:10047F0050180529E52970021529C3E529940A505A
:10048F0002A120755C00D270A120E5296002152918
:10049F007400207F037896E624FAFEE43400FFC34D
:1004AF00EC9EFCED9FFD50067800790081ECC3ECCB
:1004BF0094FFED9400400678FF790081ECEC857293
:1004CF00F0A4C5F0A2F733F87900400302050878CD
:1004DF00FF7900020508E9C313F9E813F8307C0E21
:1004EF00E9600278FFC3E81338F8E43400F9C3E891
:1004FF0094FFE99400400278FF885CD2702061027B
:10050F00A120741FF4552F4BF52FC274EB7002D23C
:10051F0074752A40307403752A0A306102A13420A1
:10052F00740353DAFE207403752B20D0F0D0E0D083
:10053F00D0D2AD43E610327901020564790302058A
:10054F0064790A020564791E020564796402056400
:10055F0079C80205647817E4D5E0FDD8FAD9F622F8
:10056F007A147B7802058B7A107B8C02058B7A0DBF
:10057F007BB402058B7A0B7BC802058BE573D5E044
:10058F0001227902E4C294D5E0FDC291D5E0FDD2FB
:10059F0091D5E0FDD294D5E0FDE920E002C2903084
:1005AF00E002C292E573D5E0FDE920E002D290307F
:1005BF00E002D2927496D5E0FDD9C9EAF8D5E0FDF4
:1005CF00D8FBDBB8C29422C37C007D0075F0000518
:1005DF00F0EA33FAEB33FB50F6EB13FBEA13FAC3F3
:1005EF00E9FFE8FEE89AF8E99BF95004EFF9EEF815
:1005FF00B3EC33FCED33FDD5F0DFEDF9ECF822E889
:10060F0089F08A20D2D4F8A9F07B0030F70B7BFF5A
:10061F00F42401F8E9F43400F9E88520F0A4ADF0F2
:10062F00F8E98520F0A4AFF0FEED2EF974003FFA43
:10063F007C04C3EA13FAE913F9E813F8DCF48BF03E
:10064F0030F70AE8F42401F8E9F43400F9E889F006
:10065F00C2D4F8A9F0227882B60403020704C3E5D6
:10066F005C9419401EE52D54067018206E367805DF
:10067F007994E7146007780A1460027812C3E54191
:10068F0098401F306E098564627569FF756A018530
:10069F002224E4F544F545F546F547F548C26E02C8
:1006AF000704D26E7994E7147013E523F43333F90A
:1006BF0013F8E9540104F9E854FE0206F8E714149C
:1006CF007014E523F4333333F913F8E9540304F9C1
:1006DF00E854FC020700E523F433333333F913F8FE
:1006EF00E954070404F9E854F8C39440F8E9940076
:1006FF00F98844894522C3E54113F9E54013F8C34E
:10070F00E54498F8E54599F9500CC3E89480E994CD
:10071F00FF401602073CC3E8947FE99400500302A0
:10072F00073C787F790002073C788079FF884989F8
:10073F004A22E5492546F8E54A3547F9854A20E436
:10074F00300701F43548FA30E709C3EA94F0401551
:10075F0002077AC3EA940F500302077A78FF79FFF2
:10076F007A0F02077A780079007AF0C3E524956151
:10077F00500AC374019524500B020798E54A20E7ED
:10078F000E020798E54A30E706884689478A4822CD
:10079F0078A5E6FAC3E54933F8E54A33F9D10EE90E
:1007AF0030E70BC3E89480E994FF4013E1D2C3E82C
:1007BF00947FE994005002E1D2787F7900E1D278FA
:1007CF008079FFE820E715C3E52398F84009C3E8CF
:1007DF00940140030207F978010207F9E8F42401B4
:1007EF002523F840030207F978FF884B2278A6E605
:1007FF00FAA847A94812060EE930E70CC3E894019E
:10080F00E994FF401602082EC3E894FFE9940050C4
:10081F000302082E78FF790002082E780179FFE98C
:10082F0020E715C3E54B98F84009C3E8940140034E
:10083F000208557801020855E8F42401254BF840C9
:10084F000302085578FF88242278FF20692879A1B0
:10085F00E76023E541601F74FF8541F0848539F01F
:0F086F00306A0375F005A4F8C5F0600278FFC386
:10087E00E895645002A864886322C3E5409440E57D
:10088E00419401E5635003140199046002F563225B
:10089E007883E6F520120F1C75E89012054675E870
:1008AE009030EDFDA8BDA9BE120FC3756E30756FE9
:1008BE0000C3740013FD7430606613FC74302CFC9E
:1008CE0074003DFDECFAEDFBC3E89AE99B4014E59C
:1008DE006E2430F56EE56F3400F56FEA2CFAEB3DC1
:1008EE00FB80E5AE6EAF6FC3E56F13F9E56E13F8DF
:1008FE00C3E913F9E813F87A03C3E913F9E813F817
:10090E00DAF7AA201A7009756E00756F0002092EAB
:10091E001AEA6008EE28FEEF39FFDAF88E6E8F6F56
:10092E002275E890227883E6FF30EDF9A8BDA9BEC6
:10093E000570C3E57094084052757000E9FA79A00D
:10094E00E76044EA7007E571601B020967C3E8952A
:10095E00716010E5715006600C140209730460F9A1
:10096E00020973E571F571C3946D401B7561C0C3C7
:10097E0094044013756180C39404400B756140C3A9
:10098E009404400375610075BB0622EFC3940160A9
:10099E001F7430601BC3E894FFE994035012C3E840
:1009AE00956EE9956F5009E561600C15610209C5F8
:1009BE00E561F460020561A861C3E524985002A8C0
:1009CE0024C3E89562400AA862E562F4600385627A
:1009DE006188258826E570B4070375BB1022743232
:1009EE0079A787F0A4C5F0A2F733F8C3E895614064
:1009FE0002A861882288248825882688642275406A
:100A0E00007541F022C2AF75C820A8CCA9CDAA3A74
:100A1E0030CF010A75C824D2AFAB3BAC3C883B89C2
:100A2E003CC3E89BF8E99C206908F9306602612412
:100A3E00417EAD3D8A3DF9EA9DFA600678FF79FF69
:100A4E004163AE3EAF3F8B3E8C3FA83BA93CC3E813
:100A5E009EF8E99FF9C3E54113FBE54013FAE82A36
:100A6E00F540E93BF54150067540FF7541FF41CB1E
:100A7E00AA40AB41AC40AD417E047F02C3EB94046F
:100A8E00400D1E1FC3EB94084005206A021E1FC3B3
:100A9E00ED13FDEC13FCDEF7C3EA9CFAEB9DFBEFC6
:100AAE006009C3E913F9E813F8DFF7EA28FAEB391E
:100ABE00FB8A408B4150067BFF8B408B41C3EB94EE
:100ACE00025002D2663069047F0341F67892E6FF47
:100ADE00C3E537948240110FC3E53794A040010F50
:100AEE00C3EF940640027F057E02E541C4540FF920
:100AFE00E541C454F0F8E540C4540F28F8C3E89E0D
:100B0E00FAE99400FB4009C3EA9402EB9400500406
:100B1E007A02E4FB6170AA40AB41EBC4FEEAC45416
:100B2E000F4EFCC3EA9CFAEB9400FBC3E813C3130D
:100B3E00F8EA28FAEB3400FB8A408B41C3EB9402AF
:100B4E004002C2667802EBC4FE7B00EAC4540F4E2C
:100B5E00FAC3EA98FA4005C3940250027A027892D8
:100B6E00E6FF3060026170855192855293D26043E8
:100B7E00E680C3E49AF8E49BF930660261FCE8FA79
:100B8E00E9FBD3E913FDE813FC88518952C3EF94B6
:100B9E00036038EF20E00DE82CF8E93DF9ECFAEDB2
:100BAE00FB020BC5E828F8E939F9C3E82402F8E995
:100BBE003400F97AFE7BFFC3EF9403400E8A538B09
:100BCE0054884D894E8C4F8D508130885389548A6C
:100BDE004D8B4E8C4F8D503069127553F07554FFFE
:100BEE00754FF07550FF7551F07552FF8130E8FA70
:100BFE00D3E813FC8851C3EF94036020EF20E00785
:100C0E00E82CF8ECFA811CE8282402F87AFEC3EFEF
:100C1E00940340088A53884D8C4F813088538A4DF7
:100C2E008C4FE568C3335002646BF5683060028107
:100C3E003A753402D26043E680E52D54066034A83E
:100C4E0040A941C3E913F9E813F8C3E913F9E8130E
:100C5E00F8306904E92440F9C2AF53E67F7591007C
:0E0C6E00C3E498F594E499F595759104D2606D
:100C7C0043E680D2AF22D264754300752000306CFD
:100C8C0003752040020CA1D26475430075204030DE
:100C9C006C0375200078017901206620E52D54063F
:100CAC006002C2647914E541C313700104F8C39463
:100CBC001440027814306904781B791B206010E50D
:100CCC0043600C306903D53404D26DA14C914205BC
:100CDC0043E59BF45440B52002A13630690908C3A2
:100CEC00E89940011881C820640A08C3E8994002B9
:100CFC0081A181C8C264C2AF53E67F759100306692
:100D0C00127594007595F8759104D26043E680D203
:100D1C00AF81A1E5417EFFC3334005C3334001FEE3
:100D2C00C3E49E759400F595A113C3E5339401506B
:100D3C000281A130640281A1D802A14A81C8C26D8E
:100D4C00C2AF53E67F759100855394855495759188
:100D5C0004854D92854E93D26043E680D2AFE52D4B
:100D6C0054066008206A020533020D88306D0D2090
:100D7C006C0A2064071581158102162C227800302C
:100D8C0064027801E53775F007A4F9E5F028F5F071
:100D9C00E9A2F013A2F113A2F213F537C394785021
:100DAC0003753778C3E53795384008D265D290D2B1
:100DBC0091D292306002A1BF854F92855093D26040
:100DCC0043E68022207D16C2AF754202C294D293B4
:100DDC00306202C292D2AF759F11020FC0C2AF75C2
:100DEC004202C294D295306202C290D2AF759F116A
:100DFC00020FC0307243207D20C2AF7542039001B8
:100E0C0034757B10D292C295306204C291C11DD24E
:100E1C0094D2AF759F21020FC0C2AF7542039001EF
:100E2C0034757B10D290C293306204C291C13DD212
:100E3C0094D2AF759F01020FC0207D17C2AF7542CF
:100E4C000390010FD292306202C291D2AF759F21F2
:100E5C00020FC0C2AF75420390010FD290306202F4
:100E6C00C291D2AF759F01020FC0207D16C2AF7523
:100E7C004204C293D295306202C291D2AF759F01E7
:100E8C00020FC0C2AF754204C295D293306202C247
:100E9C0091D2AF759F21020FC0307243207D20C2CA
:100EAC00AF754205900123757B08D291C2943062D4
:100EBC0004C290C1C3D293D2AF759F11020FC0C2AE
:100ECC00AF754205900145757B20D291C29430627A
:100EDC0004C292C1E3D295D2AF759F11020FC0200C
:100EEC007D17C2AF754205900105D291306202C2E6
:100EFC0090D2AF759F11020FC0C2AF754205900121
:100F0C0019D2913062EBC292D2AF759F11020FC011
:100F1C00207D16C2AF754206C295D294306202C2D1
:100F2C0090D2AF759F21020FC0C2AF754206C2931B
:100F3C00D294306202C292D2AF759F01020FC030C0
:100F4C007244207D20C2AF754201900145757B2013
:100F5C00D290C293306204C292E169D295D2AF753D
:100F6C009F01020FC0C2AF754201900123757B082F
:100F7C00D292C295306205C290020F8AD293D2AF40
:100F8C00759F21020FC0207D17C2AF7542019001E1
:100F9C0019D290306202C292D2AF759F01020FC07B
:100FAC00C2AF754201900105D292306202C290D25A
:100FBC00AF759F21C26522900103757B00D290D240
:100FCC0091D292C293C294C295C262227880760763
:100FDC000876070876010876040876FF0876FF087D
:100FEC007609087602087601087601788C76010875
:100FFC0076000876B40876FF0876FF0876FF087648
:10100C00030876FF0876010876FF0876250876D067
:10101C000876780876C80876040876FF0876010802
:10102C00760008767A08760A087601087601087642
:10103C00000876FF087600227887E6FFC27278886F
:10104C00C27DE630E102D27DC27E7889E630E102D3
:10105C00D27EC3EF94026008758E01D273021071B8
:0E106C00758E00C273227880E6149000809387
:10107A0078A5F67881E6149000809378A6F67886AB
:10108A00E61490008D9378A7F6789FE6F8700575B8
:10109A006B0001B8C3E8941140027811E82828F5DA
:1010AA006B256B256B28F56C256B2828F56D7886E2
:1010BA00E6F539C394025003753902789CE675380F
:1010CA00FFB402037538A0B4030375388278A3E627
:1010DA001490009A93F566120FC322227896E6FAC4
:1010EA007897E6FB7888E6B40305C3EB940EFB30E9
:1010FA007F047A007BFFC3EB9AFCC3948250027C84
:10110A00827572000572EC8572F0A4C3E5F0947DD5
:10111A0040F222D27F11E61205551205557A007B5C
:10112A00007C1012054BE55C2AFA74003BFBDCF3E9
:10113A007C04C3EB13FBEA13FADCF7FEC27F11E669
:10114A0022757C00757D00E5EF20E6037520000519
:10115A0020903FFFE520146006901DFF1460009365
:10116A0004600375EF1653D9BF7581C043FF80121F
:10117A00054675EF0643B203E5B3240220E70DF5F1
:10118A0021E5E320E0068521B343E301120FC3758D
:10119A0080FF75A40075F19175D47F75900775A5C8
:1011AA003F75F2FF75D50075A60175E241120FC3AE
:1011BA00E4F8F6D8FD756801120FD81216837898EC
:1011CA008673753001C2AF12055F12056F1205559D
:1011DA0012057612055512057D1205551217B6121B
:1011EA00055F12055F12055AC2AF757C00757D0056
:1011FA0078FA79FA308707D9FBD8F7021C0011442C
:10120A00117211E511E678988673120FC37588106A
:10121A0075890275C82475910475D84075A8227518
:10122A00B80275E690759B80759D0075D10E75BCE8
:10123A005875BB0675BA1175E880120546D2AF1209
:10124A00089E75360053DACF207E0343DA20307EBB
:10125A000343DA1043DA01C2D8C27112055FD261C0
:10126A007B037A0CE55B70077A0CDB030211F2123E
:10127A0005552070030211F2C270E55CC394024066
:10128A00E1E52F541F855E5DF55EB55DD5DAD5C201
:10129A006153DACF207E0343DA20307E0343DA102B
:1012AA00C2D8C27178A2E67008D274E52F54E0F56C
:1012BA002FC27575290012055A307409C3E529949D
:1012CA000A4002D27512054B78023074027800C3C4
:1012DA00E55C9840F0C2AF12056F12056F12056FF8
:1012EA00D2AF12055F754C0012054B788CE6C39499
:1012FA000150030213DFE530C3940150030213DFE8
:10130A00757CA5757DF1207435C3E55C94FF5003A7
:10131A000213DFC2AF120584D2AF12055AC3E55CCD
:10132A00940150EFC2AF12056F12055012056FD229
:10133A00AF12055AC3E55C94FF40E902183B7F05EA
:10134A00D27F11E612055AC2AFC27F11E6AE5CC364
:10135A00E55C947FD2AF500261EF120546C2AF122C
:10136A000584D2AFDFDA311DC3EE94057897F61201
:10137A00055F1217BE7F0AD27F11E612055AC2AF65
:10138A00C27F11E6AE5CC3E55C947FD2AF50E61231
:10139A000546C2AF12056F12055012056FD2AFDFB4
:1013AA00D6311DEE24037896F6F87997E7C394822E
:1013BA004003985006E824827897F612055F1216C1
:1013CA00D11217ED12055A11E6C3E55C94FF5002DB
:1013DA00610A02183B757C00757D00C3E55C954C7B
:1013EA004003855C4C12055A78017988E7B40302F8
:1013FA007805C3E55C98400241F2C2AF1205841237
:10140A000584120584D2AF12055F753000E4F53108
:10141A00F5320531E531F4703F0532789AE67819EC
:10142A00146012783214600D787D14600878FA140A
:10143A006003753200C3E53298401D120FC31205CE
:10144A0046153275310078998673C2AF120584D277
:10145A00AF7898867312055A120550E52A7005303E
:0F146A00740221F278012074027806C3E55C98C1
:1014790040A112055AE52A70030211F2C2AF120FF8
:10148900C3E4F522F523F524F525F526F567D2AF52
:101499007885E6C333F565E4F544F545F546F54742
:1014A900F548F570F52CF52DF53775700875BB10F5
:1014B90012054612092F30EDFDA8BDA9BEE970013C
:1014C900F8887112093375700875BB101144C2AFE1
:1014D9007561FF1209EC852261852262852263D23A
:1014E900AF7522017524017525017526018560698D
:1014F900756A017888E6B40307C27D307602D27D29
:10150900D268D269753300120F1C120F4B120A0CE4
:10151900120A13120A0C120A13120A0C120C931251
:101529000665120D89120DD0120A13120C82306E43
:10153900031207052066031208583066031208884B
:10154900120D89120DFF120A13120C93306E031239
:101559000741120D89120E76120A13120C82306E8F
:101569000312079F120D89120EA5120A13120C936A
:10157900306E031207FC120D89120F1C120A131286
:10158900092F120C82120D89120F4B120933120AFC
:101599001330692C856461856462856069756A01A7
:1015A90079187A0CC3E533994009C269D26A8A3538
:1015B9000215C9C3E55C94014003021525021634DE
:1015C900306A25206C22E535147006C26AD26BA1F7
:1015D90025F535C3E55C940140030215257888E6B5
:1015E900C394036003021634753600C3E55F9401A2
:1015F9004009856462856069756A0178FA79A4E7AA
:1016090060027803C3E55F985021307404E52A60CD
:101619001A78F0306C058564617820C3E5419850EB
:1016290002A1250536E55C6002C137753600C2AFF7
:10163900120FC37887E6FE760211447887EEF6E446
:10164900F522F523F524F525F526F565752C0075A4
:101659002D00D2AF12055A120FC378A4E66006C254
:1016690090C291C292307406E52A700221F2788DF7
:10167900E6C39401400241CF8117901A0D782012D8
:101689001713E520B4A50CA3121713E520B45A03C8
:101699000216B1757CA5757DF1120FD81216D17598
:1016A9007C00757D000216D0901A0378807B0A129F
:1016B9001713A308DBF9901A0F788C7B19121713EB
:1016C900A308DBF9901A2822C2AF12175612173352
:1016D900901A00740E121718A37409121718A3741C
:1016E90015121718901A0378807B0A121717A30886
:1016F900DBF9901A0F788C7B19121717A308DBF9FD
:10170900121769121747901A2822E493F622E64322
:101719008F01538FFDFFC3E583941C400122EF85A0
:101729007CB7857DB7F0538FFE22438F02438F012B
:10173900857CB7857DB7901A0DF0538FFC22901ADE
:101749000D74A5F118901A0E745AF118227A30798D
:10175900D07820901A40F113E520F709A3DAF7228F
:101769007A3079D0901A40E7F11809A3DAF922AB57
:1017790074A875BB01027980BB02027981BB03029F
:101789007982BB04027994BB05027983BB0602798D
:1017990086BB07027992BB08027987BB0902799C4B
:1017A900BB0A027988BB0B027989E8F7227C05120A
:1017B900055FDCFB22C2AF12056F12057612057DAB
:1017C90012058412055012056F12057612057D1255
:1017D900058412055012056F12057612057D120552
:1017E90084D2AF22C2AF12058412057D120576128A
:1017F900056F12055012058412057D120576120532
:101809006F12055012058412057D12057612056FB7
:10181900D2AF22AE74AF75C2AF12056F12056F1247
:10182900056F120550DEF2120584120550DFF8D259
:10183900AF221217BE1217B61217B6757401757555
:1018490001757600111C7C05AD5C12055FC3ED9531
:101859005C70F5C3E55C9401400AC3E55C94FF4004
:0F1869003702187E1217781216D11217BEC2AFAF
:1018780075EF161217B6DCD10576C3E576940350DA
:101888000280C21217B60575E5741490009F93F88C
:1018980008C3E57598500280A91217B61217B60545
:1018A80074C3E574940C50028095120FD81216D1A7
:0818B800C2AF75EF161217B65E
:0319FD0002114B89
:101A00000E091507070104FFFF09020101A55A018C
:101A100000B4FFFFFF03FF01FF25D078C804FF01DA
:091A200000FF0A010100FF00FFB4
:101A400023506F6C61726973546472343041232087
:101A500023424C48454C4923463333302320202031
:101A60002020202020202020202020202020202076
:101C0000C2AFC2D353D9BF7581C043B20343FF8073
:101C1000752438752503B1DC7529A5752AF175E29F
:101C20004043F18053A47F75D4FFD2877DFA7803B7
:101C300079E67C10752200752300901DE97B0675FE
:101C400024987525013087028145208708D8FBD963
:101C5000F9DCF781B7308708D8FBD9F9DCF781B711
:101C6000B19CE493A3C39A6004DDC381B7DBDBB10D
:101C70008E6002812E7B08E493FAA3B16FDBF87AC1
:101C800030B16F752200752300B18EEAFCEBFDC305
:101C9000ED94FE400EB18E8A278B28ED30E0048A49
:101CA000828B83B18E7AC270D8C3ED94FE601950D6
:101CB000CEBD002BEC600F7520007521FF7529004B
:101CC000752A000200008100A827A9280809D80465
:101CD000D90281DCB192EA89AAF281CE0D81A3C337
:101CE000ED94035053EDA2E092007AC5C3E58294CF
:101CF00000E583941C508A200010438F02438F011B
:101D00008529B7852AB7F0300029A827A92808090E
:101D1000438F01538FFDD804D902A133C3E58394C7
:101D20001C4003A3A11689AAE28529B7852AB7F02A
:101D3000A3A116538FFC817F7AC1BD030CE493A34A
:101D4000FAB153DCF8B14B817F8181AA22AB23B178
:101D50006FEBFAEA6222752608C3E52313F523E543
:101D60002213F52250066323A0632201D526EAB18F
:101D7000DCB1DC75260AEAF4200102D287300102C8
:101D8000C287B1DCC3134002C201D526EB22B19257
:101D9000EAFB208702A192308702A197752608AE40
:101DA00024AF25C3EF13FFEE13FEB1E0B1DCC3EAAD
:101DB000133087024480FA30E703632201C3E5232E
:101DC00013F523E52213F52250066323A0632201B5
:101DD000D526D9E52265236523F52222AE24AF2539
:101DE0000E0FDEFEDFFCD20122424C48656C6934E6
:071DF000373164F3300601F6
:00000001FF
